:0300000002495161
:0C49510078FFE4F6D8FD75816B024998F0
:10189A000A53746172743A20004950436F6E6E6540
:1018AA0063745245510A004950436F6E6E65637402
:1018BA00003E432C562C43432CC0E4E0EFF2E5F003
:1018CA0020D1E8EDEAEEEC49500A003E432C4D41A6
:1018DA00432C25303262583A25303262583A253044
:1018EA003262583A25303262583A25303262583AD2
:1018FA0025303262582C4D414320E0E4F0E5F10AEC
:10190A00003E432C5645522C20332E3120EEF22035
:10191A0025732025732CC2E5F0F1E8FF20495020F9
:10192A00ECEEE4F3EBFF0A004E6F762031362032FC
:10193A003030370031303A33323A3038003E432CB7
:10194A004C442C50524F473A20202020202020205F
:10195A00202020202020202020202020202020207D
:10196A00202020202020202020202020202020206D
:10197A00202020202020202020202020202020205D
:10198A00202020202020202020202020202CC4E0DD
:10199A00F2E020EFF0EEF8E8E2EAE828F4E0E9EB1A
:1019AA00290A003E2A2C312CCEF1EDEEE2EDFBE5C0
:1019BA0020EFE0F0E0ECE5F2F0FB20F1E5F2E5E201
:1019CA00EEE3EE20E8EDF2E5F0F4E5E9F1E00A00F5
:1019DA003E412C4130312C2562752E2562752E250B
:1019EA0062752E2562752C495020E0E4F0E5F1205D
:1019FA00E0E4E0EFF2E5F0E00A003E412C4130324B
:101A0A002C2562752E2562752E2562752E25627526
:101A1A002C495020E0E4F0E5F120EEF1ED2E20F122
:101A2A00E5F0E2E5F0E00A003E412C4130332C2596
:101A3A0062752E2562752E2562752E2562752C49D2
:101A4A005020E0E4F0E5F120F0E5E72E20F1E5F0A2
:101A5A00E2E5F0E00A003E412C4130342C25627563
:101A6A002E2562752E2562752E2562752CCCE0F125
:101A7A00EAE020F1E5F2E80A003E412C4130352C3B
:101A8A002562752E2562752E2562752E2562752CA6
:101A9A00D8EBFEE70A003E532C4130362C256275FE
:101AAA002CC2F0E5ECFF20EEE6E8E42E20EAE2E8BC
:101ABA00F2E0EDF6E8E820282A3130ECF1290A00B4
:101ACA003E2A2C312CC4EEEF2E20EFE0F0E0ECE5BC
:101ADA00F2F0FB20F1E5F2E5E2EEE3EE20E8EDF2CA
:101AEA00E5F0F4E5E9F1E00A003E422C5330312CEE
:101AFA002562752CC6E4E0F2FC20E7E0EFF0EEF197
:101B0A00E020F1EEE5E4E8EDE5EDE8FF20EEF22075
:101B1A00F1E5F0E2E5F0E00A003E422C5330322CC7
:101B2A002562752CCEE1ECE5ED20F120F1E5F0E23D
:101B3A00E5F0EEEC20E1E5E720EAE2E8F2E0EDF696
:101B4A00E8E90A003E422C5330332C2562752CCF2B
:101B5A00E5F0E5E7E0EFF3F1EA20EFF0E820EFEE59
:101B6A00F2E5F0E520F1E2FFE7E820F120F1E5F007
:101B7A00E2E5F0EEEC0A003E422C5330342C2562AA
:101B8A00752CCDE5F220EFE5F0E5E4E0F7E820E496
:101B9A00E8E0E3EDEEF1F2E8EAE820E220F1E5F030
:101BAA00E2E5F00A003E422C5330352C2562752CB2
:101BBA00CAE0EDE0EB20F8E8F0EEEAEEE2E5F8E064
:101BCA00F2E5EBFCEDEEE3EE20EEE1ECE5EDE00A0A
:101BDA00003E532C5330362C253032625825303291
:101BEA0062582530326258253032625825303262C6
:101BFA005825303262582C4D414320E0E4F0E5F19B
:101C0A0020F8E8F0EEEAEEE2E5F8E0F2E5EBFCEDCA
:101C1A00EEE3EE20EEE1ECE5EDE00A003E454E444F
:101C2A000A0044756D705820202020203030203062
:101C3A0031203032203033203034203035203036D5
:101C4A0020303720303820303920304120304220AF
:101C5A0030432030442030452030460A003A2000E4
:101C6A000A0044756D704420202020203030203036
:101C7A003120303220303320303420303520303695
:101C8A00203037203038203039203041203042206F
:101C9A0030432030442030452030460A00457272D5
:101CAA00206B657900526420656570726F6D0A0059
:101CBA005264204D454D0A00526420436F64650A00
:101CCA000044656275674950204F4E0A00446562B8
:101CDA0075674950204F46460A0044656275675544
:101CEA00736572204F6E0A004465627567557365A5
:101CFA0072204F46460A0044656275674D73672035
:101D0A004F6E0A0044656275674D7367204F4646F9
:101D1A000A00436F6E666967206C6F636B210A0065
:101D2A00577220656570726F6D0A0020536176657F
:101D3A0020656570726F6D210A00457272204D41EF
:101D4A004321004C6F61643E3E002A003C41303121
:101D5A003D003C4130323D003C4130333D003C4186
:101D6A0030343D003C4130353D003C4130363D0089
:101D7A004E4F4950004C494E4B434F4E545200541B
:101D8A0052415353004652004E4F4C494E4B004964
:101D9A004E49004E4F4449414700003C21003C5304
:101DAA0030313D003C5330323D003C5330333D002E
:101DBA003C5330343D003C5330353D003C533036C3
:101DCA003D00FF1D7AFF1D7FFF1D89FF1D8FFF1D2F
:0A1DDA0092FF1D99FF1D9DFF1DA43F
:06535F0001680001660078
:10531E00C2AFC28E438910758BFF758DB7D2ABD2DB
:04532E008ED2AF224A
:03001B0002482771
:10482700C0E0C083C082C0D0C2AFC28E758BFF7597
:104837008DB720060675A61E75A6E10566D202E5A8
:104847006860020568E567D3940140021567056B48
:10485700E56B540F7050D20DE56B543F701AD200C0
:10486700906F42E0601204F0E0D394B4400A908065
:10487700007480F0C2AF80FE906F3DE0600204F0EC
:104887009069B9E0600214F0906F43E0D39401405F
:1048970003E014F03005020569E56AD39464400427
:1048A700D2068002056AE565D3940140021565D2F8
:0C48B7008ED2AFD0D0D082D083D0E032BF
:10127900C291C290D2B5C20A7D027C007F07125288
:10128900B28F26E526646060097D017F6012526A8B
:10129900D20AE4FDFC7F0B1252B28F26E52630E616
:1012A900097D04E4FF12528ED20A7D017C007F077A
:1012B9001252B28F26E5267008FD7FFF12526AD2BC
:1012C9000A300A03126000C2AFC288C2A8C2AA7556
:1012D9008900124BE6906BF6E0B4FA09A3E064CEFC
:1012E9007003021379E4F52674EE2526F582E434B9
:1012F9006BF583E4F00526E526B443EC906BF674B0
:10130900FAF0A374CEF0A374CCF0906BFC740AF0DD
:10131900E4A3F0A304F0A3F0906C017403F0A374A8
:10132900CCF0906BF274FFF0A3F0A3F0E4A3F0907B
:101339006C0D7405F0E4F526E5262401FFE433FE7F
:1013490074EE2526F582E4346BF583E0FD1253052E
:101359000526E526C3944340DFE4F5A775A61E7567
:10136900A6E1907FF0F0A3F09080007480F080FEF9
:10137900D2AF906C017403F0A374CCF0E4906C00CC
:10138900F0124358EF6003123198C2B5122D8DC285
:1013990006124FBA906C0DE0C3940350037403F026
:1013A900D20AC20CC20BD293200A077E187F9A1266
:1013B900443EE4906E2DF012531EC2AFA37408F0A0
:1013C900906B6C7424F0E4A3F0906BF6E0906B6E74
:1013D900F0906BF7E0906B6FF0906BF8E0906B70AA
:1013E900F0906BF9E0906B71F0906BFAE0906B7292
:1013F900F0906BFBE0906B73F0756701E4906E2FD2
:10140900F0C207C208D2AF75A70775A61E75A6E177
:10141900125243200A19AF267E007D0312451FE4AC
:10142900FF12477D7E6C7F2DE4FB7D011245F9900B
:101439006F42E060037401F0E49069B9F0A3745558
:10144900F0A37481F0E4F569E4F56A9069B9E07094
:1014590003122808906F43E0B401119080007410C2
:10146900F0E4906F43F0D20AD20BD20C908008E0DE
:10147900F52630E405D2077410F0E52630E508D2E8
:10148900099080087420F0E52630E608D20890809B
:10149900087440F0E569D394034023908002E4F096
:1014A900908001F0908000F0E569D39406400FE444
:1014B900F569C203906E2FF0756701124FBA9080DB
:1014C900A0E07003124CDF9080B8E07003124D5910
:1014D9009080D0E07003124E38908000E070133095
:1014E9000710124069906BE9EFF0D39400400312A2
:1014F9000A1E908002E07006908000E06005D20527
:10150900021451C205E4F5699069B9E06003021457
:1015190051300912123A2A906BE9EFF0D394004046
:1015290005E0FF1253322008030216B01238B590B5
:101539006BE9EFF07003021451906C2DE054BF2455
:101549007F70030216131470030215EB2402600363
:10155900021646200A077E187FA312443E300E79F0
:10156900200376906C05E07006906C09E0605B9052
:101579006F39E0FF906C05E0B50724906F3AE0FE03
:10158900906C06E0B50618906F3BE0FE906C07E0A2
:10159900B5060C906F3CE0FE906C08E06E602B90F5
:1015A9006C09E06F7033906F3AE0FF906C0AE0B518
:1015B9000727906F3BE0FF906C0BE0B5071B906F1E
:1015C9003CE0FF906C0CE0B5070F906E2F7401F0B2
:1015D9001200217567010216B0906F3974FFF0028D
:1015E90016B0906F42E060037401F0906F31E0FF34
:1015F900906C2FE06F60030216B0906F31E004F039
:10160900E4F567906E2DF00216B03003030216B0B0
:10161900906BFCE07003021451125366D203E4F597
:1016290067906E2DF0906F3D04F0E4906F30F0A359
:10163900F0200A737E187FB112443E806A906F428F
:10164900E060037401F0300352906C2DE020E74B09
:10165900906C2FE0FF906F30E0FE6F600D906F3857
:10166900E07007EE146F703F8013906F30E004F064
:10167900906BE9E0FFD3940440031250A19068B540
:101689007482F0A37401F0906C2FE09068B7F07E3B
:10169900687FB57D03124C64021451300E09200392
:1016A90006906F3974FFF0200303021765E5677030
:1016B9006B12518BEF60207E6D7F2D906D2EE02493
:1016C90004FD124C64906F38E06003021451906C71
:1016D9000DE0F567021451906F3DE0D3943C403C16
:1016E900906F38E07036906F3D04F0906B6BE0704E
:1016F9002B12534CE4906D2DF0A37412F0906F31BE
:10170900E0906D2FF0A374FDF09069BC63A2019085
:101719006D3163A2017F1212363A809B125341EF59
:1017290060159068B57483F0E4A3F07E687FB57D99
:1017390002124C64021451E56764016003021451FA
:10174900906E2DE004F0E0C3940550030216C0C268
:1017590003E4906E2FF0120021021451E567640131
:101769006003021451906E2FE014604024FE603C27
:1017790014700302184D24046003021451E4F5693E
:10178900200E13906E2F7404F0906E2DE05401F02A
:10179900756701021451E4906E2FF0906E2D04F0DC
:1017A9007567C8906F3974FFF0021451906F39E072
:1017B900700302183C906D2D7480F0906D2F7401A8
:1017C900F0E4A3F0A304F0A37430F0A3747BF0E475
:1017D900F52674342526F582E4346DF583747DF09D
:1017E90074352526F582E4346DF583E4F0E5262485
:1017F90007906D2EF07C6F7D39906C01E0FAA3E0C3
:10180900FB7F02124A627E6D7F2DE5262409FD12B7
:101819004C64906F38E0601B125366D203E4F5679D
:10182900906E2DF0906F3D04F0E4906F30F0A3F0CE
:10183900021451906E2F7404F0906C0DE02432F56F
:10184900670214519080027410F0756703906E2D31
:10185900E06401FFF0906E2F7401F0EF7019906C45
:1018690009E06013FCA3E0FDA3E0FEA3E0FF906F95
:10187900391226BE021451906C05E0FCA3E0FDA3C9
:10188900E0FEA3E0FF906F391226BE02145180FEDC
:01189900222C
:100A1E00906C2EE0B444047F0180027F00906C2D18
:100A2E00E0B447047E0180027E00EE5F604A906B68
:100A3E00F6E0906C2FF0906BF7E0906C30F0906BCE
:100A4E00F8E0906C31F0906BF9E0906C32F0906BB6
:100A5E00FAE0906C33F0906BFBE0906C34F0906C9D
:100A6E002E7452F0906B6563A2019080A863A20170
:100A7E007F0612363A02126F906BE9E0C39408506B
:100A8E0003021278906BF6E0FF906C2FE06F60031C
:100A9E00021278906BF7E0FF906C30E06F6003020B
:100AAE001278906BF8E0FF906C31E06F60030212E9
:100ABE0078906BF9E0FF906C32E06F600302127871
:100ACE00906BFAE0FF906C33E06F60030212789047
:100ADE006BFBE0FF906C34E06F6003021278906C59
:100AEE002EE0B44415906B65E0B4FF0E63A2019046
:100AFE0080A863A2017F0612363A906F42E060032F
:100B0E007401F0906F437464F0906C2E7452F090F8
:100B1E006C2DE0646D6003020C9B7BFF7A1879BB31
:100B2E001221F47BFF7A1879D5906BF6E0F52FA39E
:100B3E00E0F530A3E0F531A3E0F532A3E0F533A301
:100B4E00E0F5341221F4752FFF75301975313275B9
:100B5E0032FF75331975343E7BFF7A19790B1221EA
:100B6E00F47BFF7A1979471221F47BFF7A1979AD5C
:100B7E001221F47BFF7A1979DA906BFCE0F52FA342
:100B8E00E0F530A3E0F531A3E0F5321221F47BFF5E
:100B9E007A1A7904906C05E0F52FA3E0F530A3E006
:100BAE00F531A3E0F5321221F47BFF7A1A793290F7
:100BBE006C09E0F52FA3E0F530A3E0F531A3E0F5E5
:100BCE00321221F47BFF7A1A7960906BF2E0F52FE6
:100BDE00A3E0F530A3E0F531A3E0F5321221F47B6A
:100BEE00FF7A1A7983906BEEE0F52FA3E0F530A330
:100BFE00E0F531A3E0F5321221F47BFF7A1A79A0E9
:100C0E00906C0DE0F52F1221F47BFF7A1A79CA123F
:100C1E0021F47BFF7A1A79F3A20EE433F52F122119
:100C2E00F47BFF7A1B7923906F38E0F52F1221F4B5
:100C3E007BFF7A1B794E906F42E0F52F1221F47BE9
:100C4E00FF7A1B7981906B6BE0F52F1221F47BFFFD
:100C5E007A1B79AFA201E433F52F1221F47BFF7AD0
:100C6E001B79DB906F32E0F52FA3E0F530A3E0F5B2
:100C7E0031A3E0F532A3E0F533A3E0F5341221F40D
:100C8E0012416D7BFF7A1C79261221F422906C2D75
:100C9E00E0644C70527E1C7F2C12443E906C35E00A
:100CAE00F527A3E0F528E4F5297D03AF28AE27123A
:100CBE00451F7E1C7F6712443EAE27AF28E4FB7DA6
:100CCE00101245F97E1C7F6A12443E74102528F5D9
:100CDE0028E43527F5270529E529C3941040CA7E57
:100CEE001C7F6A12443E22906C2DE0646C705CF5A1
:100CFE002B7E1C7F6C12443EE4F52AAF2B7E007DCA
:100D0E000312451F7E1C7F6712443EE4F529A82B73
:100D1E00E6FF74372529F582E4346CF583EFF00590
:100D2E002B0529E529B410E67E6C7F37E4FB7D1098
:100D3E001245F97E1C7F6A12443E052AE52AC394A9
:100D4E000840B87E1C7F6A12443E22906C2DE064EF
:100D5E004B7061F529741F2529F582E4346CF583F7
:100D6E00E06032741F2529F582E4346CF583E0F4DB
:100D7E006023741F2529F582E4346CF583E0FF743B
:100D8E00352529F582E4346CF583E0B50710052985
:100D9E00E529B408C09069B97432F002126F906CF4
:100DAE002D7421F0300A0302126F7E1C7FA71244AD
:100DBE003E02126F906C2DE0B4521A200A077E1C70
:100DCE007FAF12443E906C2D7472F07E6C7F2D7D41
:100DDE0008124AE622906C2DE064497045200A07FD
:100DEE007E1C7FBA12443E906C35E0F527A3E0F5E9
:100DFE0028E4F529852882852783E0FF7437252985
:100E0E00F582E4346CF583EFF00528E528700205D1
:100E1E00270529E529B480DC7E6C7F2D7D8A124A58
:100E2E00E622906C2DE064437079A3E06452704624
:100E3E00200A077E1C7FC212443E906C35E0F527D7
:100E4E00A3E0F528E4F529852882852783E493FF1E
:100E5E0074372529F582E4346CF583EFF00528E527
:100E6E0028700205270529E529B480DB7E6C7F2DCD
:100E7E007D8A124AE622906C2EE0645760030212BD
:100E8E0078906C35E0F527A3E0F52874372529F521
:100E9E0082E4346CAD82FC7B80AF28AE27125157B2
:100EAE0002126F906C2DE064446003020F42906C4E
:100EBE0035E0FF6444700302126FEFB4310CC20AC6
:100ECE007E1C7FCB12443E02126F906C35E0B43024
:100EDE000CD20A7E1C7FD712443E02126F906C35E4
:100EEE00E0B4320CD20B7E1C7FE412443E02126F31
:100EFE00906C35E0B4330CC20B7E1C7FF212443E74
:100F0E0002126F906C35E0B4340CD20C7E1D7F0152
:100F1E0012443E02126F906C35E0B4350CC20C7E5A
:100F2E001D7F0E12443E02126F906C35E0FF1200D0
:100F3E001E02126F9069B9E07013200A077E1D7FA2
:100F4E001C12443E906C2D7421F002126F9069B900
:100F5E007432F0906C2DE0FFB4510A9080007480D2
:100F6E00F0C2AF80FEEF64577045200A077E1D7FEA
:100F7E002A12443E906C36E0906BE9F0E4F529902D
:100F8E006BE9E0FFE529C39F400302126F7437251A
:100F9E0029F582E4346CF583E0FF906C35E0252969
:100FAE002464F582E4346AF583EFF0052980D0904D
:100FBE006C2DE064536003021071200A077E1D7FC2
:100FCE003512443E906BF6E0FF906A6DE06F703C18
:100FDE00906BF7E0FF906A6EE06F7030906BF8E008
:100FEE00FF906A6FE0B50724906BF9E0FF906A708E
:100FFE00E0B50718906BFAE0FF906A71E0B5070C48
:10100E00906BFBE0FF906A72E06F6016906C2D742F
:10101E0021F0300A0302126F7E1D7F4412443E02FD
:10102E00126FE4F529E4F56AAF29FE74642529F5FB
:10103E0082E4346AF583E0FD1253050529E529C3E0
:10104E0094FE40E19080007480F0C2AFE4907FF097
:10105E00F0A3F0907FFD74AAF0A374FFF0A3745573
:10106E00F080FE906C2DE0644F704C906C35E0F586
:10107E0027A3E0F528E5284527700A200A077E1DDC
:10108E007F4D12443E200A077E1D7F5412443EE4DB
:10109E00F52974372529F582E4346CF583E085282B
:1010AE0082852783F00528E528700205270529E5A6
:1010BE0029B480DE02126F906C2DE0FFB4452790AC
:1010CE0080007480F0906C35E0FDA3E0907FF0CD51
:1010DE00F0A3EDF0C2AF907FFD74AAF0A374FFF001
:1010EE00A37455F080FEEF6465600302126F906C7E
:1010FE0035E0FFA3E0907FF0CFF0A3EFF0E4F5270B
:10110E00F528D3907FF1E09528907FF0E095274069
:10111E0020E4F56A2528FFE5273401FE852882851F
:10112E002783E0FD1253050528E528700205278068
:10113E00D17E1D7F561249DDEF4E602012000390C6
:10114E006BFCEFF0120003906BFDEFF012000390BA
:10115E006BFEEFF0120003906BFFEFF07E1D7F5CD5
:10116E001249DDEF4E6020120003906C05EFF01275
:10117E000003906C06EFF0120003906C07EFF01274
:10118E000003906C08EFF07E1D7F621249DDEF4E7A
:10119E006020120003906C09EFF0120003906C0AAD
:1011AE00EFF0120003906C0BEFF0120003906C0C3A
:1011BE00EFF07E1D7F681249DDEF4E6020120003B6
:1011CE00906BF2EFF0120003906BF3EFF01200034E
:1011DE00906BF4EFF0120003906BF5EFF07E1D7F35
:1011EE006E1249DDEF4E6020120003906BEEEFF0B1
:1011FE00120003906BEFEFF0120003906BF0EFF024
:10120E00120003906BF1EFF07E1D7F741249DDEF3B
:10121E004E6008124F5D906C0DEFF0E4F529E4F589
:10122E006AE5292401FFE433FE74EE2529F582E4F4
:10123E00346BF583E0FD1253050529E529C394436C
:10124E0040DC9080007480F0C2AFE4907FF0F0A399
:10125E00F0907FFD74AAF0A374FFF0A37455F08094
:0A126E00FE7E6C7F2D7D08124AE61B
:011278002253
:10511F00AE07EEC39430400BEED394395005EE2416
:10512F00D0FF22EEC39461400BEED394665005EE90
:10513F0024A9FF22EEC39441400BEED394465005B1
:08514F00EE24C9FF22AF062285
:1052EB00906B64E004F07006906B63E004F0906BDD
:0A52FB0063E0FEA3E0FF1252CF2291
:100003001252EB12511FEFC454F0FEC0061252EB12
:0800130012511FD0E02FFF2263
:104F5D00E4907080F01252EB907081EFF0C39430BA
:104F6D004018E0FFD394395011907080E024BCF5C7
:104F7D0082E43469F583EFF08011907080E024BCF9
:104F8D00F582E43469F583E4F0800C907080E004E0
:104F9D00F0E0D3940840BE752F00753000753100D8
:0C4FAD00E4F5327B017A6979BC123711FF
:014FB90022D5
:0449DD008E2C8F2D60
:1049E100906B63E4F0A374FFF01252EBEF606EF48E
:1049F100606B852D82852C83E493B507EC752E01C0
:104A0100E52D252EF582E4352CF583E49360259080
:104A11006B64E0252EFF906B63E03400FE1252CFF1
:104A2100E52D252EF582E4352CF583E493B50704B5
:104A3100052E80CCE52D252EF582E4352CF583E479
:104A41009370A6E52E24FFFFE434FFFE906B64E033
:104A51002FF0906B63E03EF07E007F0122E4FEFFC9
:014A61002232
:104358007E1D7FA51249DDEF4E70037F01227E1D71
:104368007FA81249DDEF4E600C1252EBEF24D024E7
:10437800FF920E8002D20E7E1D7FAE1249DDEF4EF7
:10438800600C1252EBEF24D0906F38F08005E49067
:104398006F38F07E1D7FB41249DDEF4E600C12526B
:1043A800EBEF24D0906F42F08005E4906F42F07EEE
:1043B8001D7FBA1249DDEF4E600C1252EBEF24D08C
:1043C800906B6BF08005E4906B6BF07E1D7FC012E4
:1043D80049DDEF4E600C1252EBEF24D024FF92011E
:1043E8008002C201906BF663A201906F3263A20152
:1043F8007F0612363A30013B7E1D7FC61249DDEF3B
:104408004E6030120003906F32EFF0120003906F8D
:1044180033EFF0120003906F34EFF0120003906F47
:1044280035EFF0120003906F36EFF0120003906F33
:0644380037EFF07F0022C7
:10319800C201E4906F42F0D20EC204906F38F090F2
:1031A8006B6BF0906BF663A201906F3263A2017FA4
:1031B8000612363AE4F527E52775F003A424CCF582
:1031C80082E4341DF583E493FB740193FA7402934B
:1031D800F91224EE700302338AE4F528F529FD7408
:1031E800E42DF582E43469F583E0FF70030233854A
:1031F800E52775F003A424CCF582E4341DF583E4B7
:1032080093FB740193FA740293F9852882758300FD
:10321800122507FEEFB50608752901052802338136
:10322800E5297003023381EE600302337CE527242D
:10323800FE602814700302336414700302336814A8
:1032480070030233701470030233742405600302A0
:103258003385906F427401F0023385D20174E42DF6
:10326800F582E43469F583E0FF642D700302338549
:1032780012511FEFC454F0FC74E52DF582E4346953
:10328800F583E0FF12511FEF2C906F32F074E62D9A
:10329800F582E43469F583E0FF12511FEFC454F05E
:1032A800FC74E72DF582E43469F583E0FF12511FC1
:1032B800EF2C906F33F074E82DF582E43469F583D0
:1032C800E0FF12511FEFC454F0FC74E92DF582E4BD
:1032D8003469F583E0FF12511FEF2C906F34F074BE
:1032E800EA2DF582E43469F583E0FF12511FEFC43B
:1032F80054F0FC74EB2DF582E43469F583E0FF1299
:10330800511FEF2C906F35F074EC2DF582E4346981
:10331800F583E0FF12511FEFC454F0FC74ED2DF556
:1033280082E43469F583E0FF12511FEF2C906F3669
:10333800F074EE2DF582E43469F583E0FF12511F35
:10334800EFC454F0FC74EF2DF582E43469F583E0A2
:10335800FF12511FEF2C906F37F08021D204801D8F
:10336800906F387401F08015C20E8011906B6B74E9
:1033780001F08009E4F529F5280D0231E705270257
:0233880031BF53
:01338A002220
:10501300906E2EE0C3947C503D906E2EE0FE04F023
:10502300746C2EF582E4346BF583EFF0BF0A27909E
:105033006E2EE0FF04F0746C2FF582E4346BF5837D
:10504300E4F0906E2EE0FF124B68906E2E7408F021
:07505300906B6DE004F022F8
:104FBA009080007480F0906BEE63A201F583F58215
:104FCA0063A2017F0812363A906BF663A2019080C1
:104FDA008863A2017F0A12363A908092E4F0A374A1
:104FEA0032F0A37401F0906C00E0FF9080B1F09071
:104FFA0080E1EFF09080957455F0A3F090800074F2
:09500A0001F09080097470F0229D
:104CDF00908009E04410F09080A0E0706C9080A16B
:104CEF007482F09080A874FFF0A3F0A3F0A3F07F7C
:104CFF00039080AEEFF07FCBA3EFF07F039080ACFB
:104D0F00EFF0A374CBF09080007402F090707212E9
:104D1F0026CA00000000907072E0908040F0907002
:104D2F0073E0908041F0907074E0908042F090704A
:104D3F0075E0908043F0A3E4F0A3F0A3F0A3F0900C
:094D4F008018F0A3F0A3F0A3F01A
:014D58002238
:104E3800908009E04440F09080D17482F0906C0139
:104E4800E0FF9080DEF0906C02E0FF9080DFF09051
:104E580080027402F09070761226CA00000000905A
:104E68007076E0908058F0907077E0908059F090DC
:104E78007078E090805AF0907079E090805BF0A3B1
:104E8800E4F0A3F0A3F0A3F0908030F0A3F0A3F037
:024E9800A3F085
:014E9A0022F5
:104D5900908009E04420F09080B8E0706C9080B9B0
:104D69007482F07F039080C6EFF07FCDA3EFF07FD0
:104D7900039080C4EFF0A374CDF09080C074FFF06D
:104D8900A3F0A3F0A3F09080017402F090707A125E
:104D990026CA00000000907076E090804CF0907078
:104DA90077E090804DF0907078E090804EF09070B0
:104DB90079E090804FF0A3E4F0A3F0A3F0A3F09082
:094DC9008024F0A3F0A3F0A3F094
:014DD20022BE
:104A62008C278D28A907EAFDE975F018A424ACFF6C
:104A7200E5F034808F82F583EDF0EBFDE975F018F7
:104A8200A4FFAEF024ACFBEE34808B82F583A3ED61
:104A9200F08528828C83E0FDEF24A8FFEE3480FEAF
:104AA2008F82F583EDF08528828C83A3E08F828E3E
:104AB20083A3F0852882852783A3A3E0FDE975F00F
:104AC20018A424A8FFE5F03480FE8F82F583A3A307
:104AD200EDF08528828C83A3A3A3E08F828E83A32B
:044AE200A3A3F02278
:064AE6008D2CAB07AA06AF
:104AEC00907072E0FCA3E0FDA3E0FEA3E0F5308E35
:104AFC002F8D2E8C2DAE02AF038E838F8263A2017D
:104B0C00E52F540744C0F58385308263A201AF2C96
:104B1C001236A3908000E020E5F9E4FCFDFEE530C0
:104B2C00252CF530EE352FF52FED352EF52EEC35F9
:104B3C002DF52D908040E52DF0A3E52EF0A3E52F6B
:104B4C00F0A3E530F09080007420F0AF30AE2FADC4
:0B4B5C002EAC2D9070721226BEAF2C04
:014B6700222B
:064C64008D27AB07AA0634
:104C6A00907076E0FCA3E0FDA3E0FEA3E0F52B8EB6
:104C7A002A8D298C28AE02AF038E838F8263A2010C
:104C8A00E52A540744D0F583852B8263A201AF2716
:104C9A001236A3E4FCFDFEE52B2527F52BEE352A7B
:104CAA00F52AED3529F529EC3528F528908058E5BF
:104CBA0028F0A3E529F0A3E52AF0A3E52BF09080DC
:104CCA00027420F0AF2BAE2AAD29AC289070761270
:044CDA0026BEAF271C
:014CDE0022B3
:02477D008F2883
:10477F00908001E030E5037F002290707AE0FCA387
:10478F00E0FDA3E0FEA3E0F52C8E2B8D2A8C299063
:10479F006F3263A201E52B540744C8F583852C8241
:1047AF0063A2017F061236B9E52C2406F52CE435F9
:1047BF002BF52BE4352AF52AE43529F529906E30AF
:1047CF0063A201E52B540744C8F583852C8263A2AD
:1047DF0001AF281236B9E4FCFDFEE52C2528F52C97
:1047EF00EE352BF52BED352AF52AEC3529F52990E9
:1047FF00804CE529F0A3E52AF0A3E52BF0A3E52CE7
:10480F00F09080017420F0AF2CAE2BAD2AAC299024
:07481F00707A1226BEAF28DB
:01482600226F
:104069009081E0E0F527052705270527052705277E
:1040790005270527052705270527908010E0F52A3C
:10408900A3E0F52BA3E0F52CA3E0F52D9081E1E069
:10409900F5270527052705270527052705270527C7
:1040A900052705270527908014E0F52EA3E0F52FB5
:1040B900A3E0F530A3E0F531E530B52C08E531B5DD
:1040C9002D037F0022E4F527E530540744E0F5830A
:1040D90085318263A201906C2D63A2017F0812369B
:1040E900D1906C2F63A201906B6563A2017F0612C8
:1040F900363A906C2DE0F528A3E0F529E4F52790F0
:104109006C2DE0702AA3E024F8F527E53054074424
:10411900E0F58385318274082582F582E43583F5DB
:104129008363A201906C2D63A201AF271236D1AE31
:1041390028E4FCFDE5312529F531E5303EF530ED82
:10414900352FF52FEC352EF52E908014E52EF0A3A2
:10415900E52FF0A3E530F0A3E531F090800074403D
:03416900F0AF278D
:01416C002230
:1038B5009081E6E0F5270527052705270527052734
:1038C50005270527052705270527908028E0F52AE0
:1038D500A3E0F52BA3E0F52CA3E0F52D9081E7E01F
:1038E500F527052705270527052705270527052783
:1038F50005270527052790802CE0F52EA3E0F52F59
:10390500A3E0F530A3E0F531E4F527E530B52C0A61
:10391500E531B52D05C208023A0FE530540744F0EC
:10392500F58385318263A201906C2D63A2017F0826
:103935001236D1906C2DE0F528A3E0F529E529454F
:103945002870099080027410F07F0022906F39E092
:10395500FFF4602D906C2FE06F7076906F3AE0FF6A
:10396500906C30E06F706A906F3BE0FF906C31E0D7
:103975006F705E906F3CE0FF906C32E06F6022806C
:1039850050906C2FE0906F39F0906C30E0906F3A6A
:10399500F0906C31E0906F3BF0906C32E0906F3CB2
:1039A500F0906C2DE0702AA3E024F8F527E530545B
:1039B5000744F0F58385318274082582F582E43564
:1039C50083F58363A201906C2D63A201AF271236A4
:1039D500D1AE28E4FCFDE5312529F531E5303EF58C
:1039E50030ED352FF52FEC352EF52EAF2DAE2CAD58
:1039F5002BAC2AAB31AA30A92FA82ED312268D4085
:103A0500099080027410F07F002290802CE52EF042
:103A1500A3E52FF0A3E530F0A3E531F09080027423
:043A250040F0AF2797
:013A2900227A
:103A2A009081E3E0F52705270527052705270527C0
:103A3A000527052705270527052790801CE0F52A75
:103A4A00A3E0F52BA3E0F52CA3E0F52D9081E4E0AB
:103A5A00F52705270527052705270527052705270C
:103A6A00052705270527908020E0F52EA3E0F52FEE
:103A7A00A3E0F530A3E0F531E4F527E530B52C0AEB
:103A8A00E531B52D05C209023B75E530540744E816
:103A9A00F58385318263A2019068B963A2017F0E22
:103AAA001236E79068B9E0F528A3E0F5299068C1D5
:103ABA00E0FFF46045906F32E0FEEF6E706EA3E0B7
:103ACA00FF9068C2E06F7064906F34E0FF9068C343
:103ADA00E06F7058906F35E0FF9068C4E06F704CEB
:103AEA00906F36E0FF9068C5E06F7040906F37E0E6
:103AFA00FF9068C6E06F60048032D2D99068B9E05E
:103B0A00702AA3E024F2F527E530540744E8F58348
:103B1A00853182740E2582F582E43583F58363A2AA
:103B2A00019068B963A201AF271236E7AE28E4FC18
:103B3A00FDE5312529F531E5303EF530ED352FF536
:103B4A002FEC352EF52EAF2DAE2CAD2BAC2AAB318A
:103B5A00AA30A92FA82ED312268D5006E52945286A
:103B6A0070099080017410F07F0022908020E52E69
:103B7A00F0A3E52FF0A3E530F0A3E531F090800142
:053B8A007440F0AF27BC
:013B8F002213
:04443E008E2D8F2E02
:10444200907072E0FCA3E0FDA3E0FEA3E0F5348EE1
:10445200338D328C31E534FFE5335407FEE42FF51A
:1044620030EE34C0F52F853082F5837423F00530A9
:10447200E5307002052F532FC7F582852F83740A0A
:10448200F00530E5307002052F532FC7906BF663AD
:10449200A201852F8385308263A2017F061236A393
:1044A20074062530F530E4352FF52F852D83852EC2
:1044B2008263A201852F8385308263A2011236872F
:1044C200908000E020E5F9E4FCFDFE907072E0F8D7
:1044D200A3E0F9A3E0FAA3E02FFFEE3AFEED39FDE7
:1044E200EC38FCEF2408FFE43EFEE43DFDE43CFC36
:1044F2009070721226BE907072E0908040F09070C0
:1045020073E0908041F0907074E0908042F090707F
:0C45120075E0908043F09080007420F071
:01451E00227A
:0645F9008E2D8F2E8D2F88
:1045FF00907072E0FCA3E0FDA3E0FEA3E0F5358E22
:10460F00348D338C32E535FFE5345407FEE42FF556
:10461F0031EE34C0F530853182F5837423F00531E6
:10462F00E531700205305330C7F582853083EBF0EA
:10463F000531E531700205305330C7906BF663A238
:10464F000185308385318263A2017F061236A37400
:10465F00062531F531E43530F530852D83852E82F1
:10466F0063A20185308385318263A201AF2F123699
:10467F00A3908000E020E5F97408252FF52FFFE4C3
:10468F00FCFDFEE5352FF535EE3534F534ED3533DC
:10469F00F533EC3532F532908040E532F0A3E53357
:1046AF00F0A3E534F0A3E535F09080007420F0AF6F
:0D46BF0035AE34AD33AC329070721226BEB1
:0146CC0022CB
:024B68008F407C
:104B6A00907072E0FCA3E0FDA3E0FEA3E0F5448EA2
:104B7A00438D428C41E544FFE5435407FEE42FFF91
:104B8A00EE34C0906B6C63A201F5838F8263A2013D
:104B9A00AF401236A3908000E020E5F9E4FCFDFE68
:104BAA00E5442540F544EE3543F543ED3542F542FB
:104BBA00EC3541F541908040E541F0A3E542F0A390
:104BCA00E543F0A3E544F09080007420F0AF44AED2
:0B4BDA0043AD42AC419070721226BE49
:014BE50022AD
:06451F008E2C8F2DAB0570
:10452500907072E0FCA3E0FDA3E0FEA3E0F5338EFE
:10453500328D318C30E533FFE5325407FEE42FF53B
:104545002FEE34C0F52E852F82F5837423F0052FC9
:10455500E52F7002052E532EC7F582852E83EBF0CD
:10456500052FE52F7002052E906BF663A201852EAF
:1045750083852F8263A2017F061236A37406252F39
:10458500F52FE4352EF52E532EC7E52C852F828584
:104595002E83F0052FE52F7002052E532EC7F582C9
:1045A500852E83E52DF0052FE52F7002052E532E60
:1045B500C7908000E020E5F9E533240AF533E435BA
:1045C50032F532E43531F531E43530F5309080405F
:1045D500E530F0A3E531F0A3E532F0A3E533F09043
:1045E50080007420F0AF33AE32AD31AC30907072D4
:0345F5001226BECD
:0145F80022A0
:1052CF00E5D220E0FBC2AF438E2075D2028F828ED3
:0B52DF0083E0FFE4F5D2538EDFD2AF76
:0152EA0022A1
:10530500E5D220E0FBC2AF43D2028F828E83EDF05F
:0953150075D25063D250D2AF22D0
:104BE600E4FDED2401FFE433FE1252CF74EE2DF501
:104BF60082E4346BF583EFF00DBD3FE6E4FDED2472
:104C06007FFFE433FE1252CF74E42DF582E434695B
:104C1600F583EFF074E42DF582E43469F583E070F2
:104C26001B74E42DF582E43469F5837420F074E591
:104C36002DF582E43469F583E4F080040DBD80BE71
:104C4600E4906A63F0FDEDFF7E001252CF74642D8E
:0D4C5600F582E4346AF583EFF00DBDFEE950
:014C6300222E
:025157008B2C9F
:10515900A2AF921EC2AF85A22D53A2FE8E838F826B
:1051690005A28C838D8274091236FFE52C53A2FEA9
:1051790043A22012370153A2DF852DA2A21E92AFAE
:01518900FF26
:01518A002202
:1052B200A2AF921EC2AF8C838D82EF1236FF43A241
:0C52C2002012370153A2DFA21E92AFFFA2
:0152CE0022BD
:02526A008F278C
:10526C00A2AF921EC2AFE4F5838D8274061236FF94
:10527C00E52743A22012370153A2DFA21E92AF7F73
:01528C000120
:01528D0022FE
:02528E008F2768
:10529000A2AF921EC2AFE4F5838D82740A1236FF6C
:1052A000E52743A22012370153A2DFA21E92AF7F4F
:0152B00001FC
:0152B10022DA
:10355F00A907E7FFA805EF93C3966008403B74FCEB
:10356F002FFF80F00F08EF93C3966008402B74FB7A
:10357F002FFF80E00F08EF93C3966008401B74FA8B
:10358F002FFF80D00F08EF93D3966008400B74F98C
:10359F002FFF80C01F1F1F1F1FEF54FEF80303F7DD
:1035AF00E893FC08E893FD08E893FE08E893FF22F0
:1035BF0009E993C39D6008402974FB29F980F1093B
:1035CF00E993C39E6008401A74FA29F980E209E969
:1035DF0093D39F6008400B74F929F980D3191919F7
:1035EF001919E9C313C313FF22740093F8ECC3989E
:1035FF004024701F740193F8EDC398401970147430
:0E360F000293F8EEC398400E7009740393F80E
:10361D00EFC39840037F00227F0122EDF8E6F0080A
:10362D00A3DFFA22EDF8E0F608A3DFFA22E0A363A8
:10363D00A201F0A363A201DFF475A20022E0A3634F
:10364D00A201F0A363A201E0A363A201F0A363A210
:10365D0001E463A201F0A363A201DFE175A20022E0
:10366D00E0A363A2016DFE936CFDEE058393FC1543
:10367D008363A201DFEA75A200227F00E493A363B6
:10368D00A201F00F600CA3E583C2E3F58363A201F1
:10369D0080EA75A20022E0A363A201F0A3E583C234
:1036AD00E3F58363A201DFEE75A20022E0A363A21E
:1036BD0001F0A3E583C2E4D2E3F58363A201DFEC5D
:1036CD0075A20022E583C2E3F583E0A363A201F0B6
:1036DD00A363A201DFEE75A20022E583C2E4D2E36B
:1036ED00F583E0A363A201F0A363A201DFEC75A251
:1036FD000022F922C002C004C00612FFF0D006D08D
:04370D0004D00222C0
:1048C3000A536572763A004572724C656E210A008E
:1048D300205544502054696D654750530A00200AFF
:1048E300444154414752414D3A20002043414E2018
:1048F30054696D654750530A0020547261737353B2
:10490300656E644552520A000ACEF8C4EBE8EDFB2B
:1049130043414E210A000A45727241647243414E7B
:104923003A000A00205265496E69742043414E0AD9
:10493300002043414E283029203E20544F210A00B5
:0E49430020545520300A0020545520310A001F
:03001E00E4FF22DA
:10521B00C2A9438902758C48758A4875D90475DB18
:10522B004875DC4875DD4875DE48E4F5E9F5F9D2DB
:08523B00D9C2DAD28CD2DE22C6
:1051ED00C2D9906F58E07013E5E92419F5EB30D76B
:1051FD0006E5F904F5FB2285F9FB22E5E924C8F55E
:0E520D00EB30D706E5F904F5FB2285F9FB220C
:10505A00C2D9906F58E0702C302B16E5E92432F54E
:10506A00EB30D707E5F904F5FB800385F9FBC22B82
:10507A0022E5E92405F5EB30D706E5F904F5FB222C
:10508A0085F9FB22E5E92432F5EB30D706E5F90488
:07509A00F5FB2285F9FB2262
:1052430012521B906F58E0C394645006124DD31250
:1052530051ED120022D22AE4F556907070F0F54514
:07526300F55AC22BF5582299
:1050A100EF24FCF545200A127E487FC312443E7E60
:1050B1006C7F31E4FBAD451245F9E545D3940D40D4
:1050C10010200A077E487FCA12443EE4F545D228E3
:1050D10022906C3163A20190706063A201AF45120E
:0550E100363AC228224E
:0F533200D3EF6480948D5006E55A70028F5A2293
:1028080020D9030228E5202A030228E5E55A605268
:102818009068B9540FFF7D47123631E5476401705F
:102828001E9068C1E0B4FF0ED22C200A127E487FA9
:10283800D312443E8009302C06E4F55A0228E512EA
:1028480051ED124E9B200A077E487FE112443E203C
:102858000A0B7E687FB9E4FBAD5A1245F9E4F55AD4
:10286800807BE5456043907064E02405F527D394A8
:102878000D4007E4F545D2288063907060E5275441
:102888000FFF7D47123631E54730E702D22BE54787
:10289800B40109302C06E54A64016003124E9B120C
:1028A80051EDE4F545D2288034E557601E906F4419
:1028B800540FFF7D47123631E547B40103202C033E
:1028C800124E9B1251EDE4F557801220100C906FB8
:1028D80058E0C394645003124EFD1251ED123B9020
:1028E8008F27EF70030229AC12505AE4F558E547D8
:1028F800B4010CD22C200A077E487FEE12443EE534
:1029080059C394C8502D30032AE547B4420DE54A0F
:10291800B40208906B6BE06401601874592559F58E
:1029280082E4346FF583E5272559F5597D47AF27AC
:10293800123628300121E54720E71C906E307D478C
:10294800AF27123628AF2712477DEF700A200A07F3
:102958007E487FFC12443EE54754817047E527D303
:10296800940D400C200A3D7E497F0B12443E803472
:10297800E549D394074028200A2A7E497F19124442
:102988003E9069BC7D47AF271236287E697FBCE43C
:10299800FBAD271245F97E497F2512443E8005AFDD
:1029A80027122AD9300D2C90661AE0C394FA5003E6
:1029B800E004F030001B906F58E0C3946450120597
:1029C80058E55894F0400A9080007480F0C2AF80B7
:1029D800FEC20D200203022AD3E5566031D39401CA
:1029E800400415568028907070E004F0E0D39403FA
:1029F800400D200A077E497F2712443E1252432089
:102A08000A077E497F3412443EE4F556D22A30291B
:102A180043E557703F906F4404F0A37408F0A37423
:102A280080F0A37401F0A37406F090705BE0906FDF
:102A380049F090705CE0906F4AF090705DE0906FA4
:102A48004BF090705EE0906F4CF0E4A3F0A3F0754B
:102A5800570BC229302772907059E07035E55770CE
:102A680031906F447442F0A37408F090705AE0906B
:102A78006F46F090705FE0906F47F0A37401F075B7
:102A88005706200A077E497F4312443E907059E05A
:102A980004F0907059E06402702FE557702B906F26
:102AA800447402F0A37408F090705AE0906F46F0F6
:102AB800A3F0A37401F0755706200A077E497F4AE0
:102AC80012443E907059E004F0C202120026C2007F
:012AD80022DB
:10518B00E559602CE4906D2DF0A3E559F0906F314B
:10519B00E0906D2FF0A37419F0906F5963A20190FA
:1051AB006D3163A201AF5912363AE4F5597F0122F2
:0351BB007F002250
:0B534100302805C2287F01227F0022D7
:0100210022BC
:06536600E4F559F54522B3
:0A534C00E49069BCF0A3F0A3F02286
:1051BE002043616E457247495400200A00457272C1
:1051CE004C656E43616E21000A002043616E45728C
:0F51DE0072434821000A20526571457272210008
:103B9000E59B541F6020200A1A7E517FBE12443ECE
:103BA000E59B541FFF7E007D0312451F7E517FC899
:103BB00012443EE4F59BE5BA30E010E4F5B375B18C
:103BC00080F5B2D22AF556907070F0E5CFF470030C
:103BD000023CE5752901E4F528E5CFF45529700389
:103BE000023CD3E528C454F0F5B1E5B2547F64201B
:103BF0006003023CA4E5B3540FF54B85BC47E5BD1B
:103C0000541FFF131313541FFFE5BD54E044184F16
:103C1000F548E5BDC43354E0FFE5BE131313541F4C
:103C20004FF549E5BEC43354E0FFE5BF1313135409
:103C30001F4FF54A85A34C85A34D85A34E85A34F01
:103C400085A35085A35185A35285A353E4F5B220E3
:103C5000100CE547547EB5470575B350800375B326
:103C6000D0E54B700AE547547EB547037F0022300C
:103C70001008E54730E7037F0022E54BD394084066
:103C80001D200A177E517FCB12443EAF4B7E007D34
:103C90000312451F7E517FD612443E7F0022E54B22
:103CA0002405FF22E5B2549F6023200A207E517F25
:103CB000D812443EAFB27E007D0312451FAFB37EE3
:103CC000007D0312451F7E517FD612443EE4F5B2BB
:103CD00075B3D0E52925E0F5290528E528C3940822
:073CE0005003023BD97F00F5
:013CE70022BA
:104E9B00906F58E0C39464505675B180E4F5B3F548
:104EAB00B28547BCE549C4135407FFE54854E04FAE
:104EBB00F5BDE54933333354F8FFE54AC4135407C2
:104ECB004FF5BEE54A33333354F8F5BF854CA38514
:104EDB004DA3854EA3854FA38550A38551A3855222
:104EEB00A38553A3E54B540F2450F5B375560AC253
:024EFB002A2269
:104EFD0075B190E5B220E613200A107E517FE312C2
:104F0D00443EAFB27E007D0312451FE4F5B3F5B20A
:104F1D00748D2517F582E43461F583E0F5BCE4F575
:104F2D00BD748E2517F582E43461F583E0FF3333CC
:104F3D003354F8F5BE75BF7805170517748D251711
:104F4D00F582E43461F583E07002F51775B35022F4
:09535600EF6003C29622D29622F8
:104DD30043AB01C2E8C2EAE4FFEFC454F0F5B1C348
:104DE300EF64809488500575B3D08003E4F5B3E491
:104DF300F5B2F5BCF5BDF5BEF5BFF5C4F5C5F5C611
:104E0300F5C7F5A3F5A3F5A3F5A3F5A3F5A3F5A3BB
:104E1300F5A30FBF0EC3906F58E0FF25E0F5B475FF
:104E2300B50C75B66C75A11275AB0275C13E75C331
:044E3300FF75C20342
:014E37002258
:10338B000000000000000000000000000000000032
:10339B003FF3630041D5E80043B71B8045984F00CE
:1033AB0047798280495C07804B3D3B004D1E6E8008
:1033BB004EFFA20050E2270052C35A8054A48E0045
:1033CB005685C180586846805A497A005C2AAD8080
:1033DB005E0BE1005FEE660061CF998063B0CD00BC
:1033EB0065920080677485806955B9006B36EC80F7
:1033FB006D1820006EFAA50070DBD880000000006D
:10340B000028DE80004DC8800076A700009E3400A7
:10341B0000C7123000EE9F8001177E0001405C80D8
:10342B000167E9800190C80001B8550001E13380C4
:10343B00000000000028DE80004F1A000077F880A3
:10344B00009F858000C8640000EFF1000118CF8059
:10345B000141AE0001693B000192198001B9A680C0
:10346B0001E2850000000000000151800002A30072
:10347B000003F48000054600000697800007E90072
:10348B0000093A80000A8C00000BDD80000D2F0034
:10349B00000E8080000FD2000011238000127500F7
:1034AB000013C68000151800001669800017BB00BA
:1034BB0000190C80001A5E00001BAF80001D01007C
:1034CB00001E5280001FA4000020F5800022470040
:1034DB00002398800024EA0000263B8000278D0003
:1034EB000028DE800000000000000E1000001C20F1
:1034FB0000002A30000038400000465000005460A5
:10350B00000062700000708000007E9000008CA0B4
:10351B0000009AB00000A8C00000B6D00000C4E0C4
:10352B000000D2F00000E1000000EF100000FD20D1
:10353B0000010B30000119400001275000013560DC
:10354B0000014370000151801F1C1F1E1F1E1F1FF7
:04355B001E1F1E1FF2
:103F4600E55B25E025E0248BF582E43433F5831226
:103F5600269E8F648E638D628C61E55B54037028A8
:103F6600E56025E025E02437F582E43434F5831254
:103F7600269EEF2564F564EE3563F563ED3562F54F
:103F860062EC3561F5618026E56025E025E02403D5
:103F9600F582E43434F58312269EEF2564F564EE4B
:103FA6003563F563ED3562F562EC3561F561E55D26
:103FB60025E025E0246BF582E43434F58312269E51
:103FC600EF2564F564EE3563F563ED3562F562EC75
:103FD6003561F561E55EC3940C402AE56424C0F5BD
:103FE60064E56334A8F563E43562F562E43561F5AA
:103FF60061E55E24F4FF7E007C0E7D10122534AA56
:1040060006AB07800FAF5E7E007C0E7D1012253456
:10401600AA06AB07AE02E4FCFDE5642BF564E56396
:104026003EF563ED3562F562EC3561F561E55F7588
:10403600F03CA4FFAEF0E4E5642FF564E5633EF5DD
:1040460063ED3562F562EC3561F561E4FEE5642504
:104056005CF564EE3563F563ED3562F562EC35616A
:02406600F56102
:014068002235
:103CE800907088E0F55B25E025E0248BF582E434CC
:103CF80033F583E55BD3941F501DAF64AE63AD62AB
:103D0800AC611235F8EF700F74042582F582E43542
:103D180083F583055B80DC74FC2582F58274FF35AE
:103D280083F583AF821226AEC3E5649BF564E56331
:103D38009AF563E56299F562E56198F561155BE5C9
:103D48005B14907088F0E55B5403700590343B80F9
:103D5800039034077560307F607D6112355FA80479
:103D6800A905AA06C3E5649FF564E5639AF563E5CA
:103D78006299F562E56198F561056090346FAF640A
:103D8800AE63AD62AC617B007A00797C1235BF8F7F
:103D98005DEF25E025E0246FF582E43434F58312E5
:103DA80026AEC3E5649BF564E5639AF563E562991D
:103DB800F562E56198F561055D9034EFAF64AE6337
:103DC800AD62AC617B007A00795C1235BF8F5EEF23
:103DD80025E025E024EFF582E43434F5831226AE9D
:103DE800C3E5649BF564E5639AF563E56299F5625A
:103DF800E56198F561AE63AF647C007D3C122546B1
:103E08008D5CAE63AF647C007D3C1225468E638F6B
:053E18006485645F22D7
:101DE40042415544004D4158420052545300444529
:101DF4004C4159005452414E5A0043414E004B50FD
:101E040000544F52455000003E2A2C312CCFE0F0B4
:101E1400E0ECE5F2F0FB20F3EFF0E0E2EBFFFEF99B
:101E2400E5E3EE20EAEEEDF2F0EEEBEBE5F0E02098
:101E3400CACF20C8F1E5F2FC0A003E4C2C6B3031CD
:101E44002C25732C43EAEEF0EEF1F2FC20EDE020B9
:101E5400F8E8EDE52043414E2C30202D203530307C
:101E6400EAE1283530EC292C31202D203530EAE107
:101E740028353030EC290A0030202D20353030EA66
:101E8400E1283530EC290031202D203530EAE128D5
:101E9400353030EC29003E532C6B30322C256275E2
:101EA4002CCCE0EAF12E20E0E4F0E5F120E1EBEEC9
:101EB400EAE020D2D128302D38290A003E532C6B79
:101EC40030332C2562752CCCE0EAF12E20E0E4F0CE
:101ED400E5F120E1EBEEEAE020D2C8D228302D383B
:101EE400290A003E532C6B30342C2562752CCCE02F
:101EF400EAF12E20E0E4F0E5F120E1EBEEEAE02067
:101F0400D2D328302D38290A003E422C6330312C9C
:101F14002562752CC2F2EEF0E8F7EDFBE920EAEE5B
:101F2400EDF2F0EEEBEBE5F020EDE020F8E8EDE586
:101F34000A003E2A2C312CCFE0F0E0ECE5F2F0FB75
:101F440020EFF0EEF2EEEAEEEBE020CCDDCA203832
:101F540037302D352D31303120EFEE20EFEEF0F219
:101F6400F32052533233320A003E432C5061723212
:101F74002C20253034752F253034752F25303475B9
:101F84002F253034752CCDE0F7E0EBFCEDFBE5209C
:101F9400E0E4F0E5F1E020D2D12FD2C8D22FD2C8AC
:101FA400C82FD2D32028F4E8EAF1E8F0EEE2E0ED1D
:101FB400EDFBE5290A003E4C2C6B30352C256C7565
:101FC4002CD1EAEEF0EEF1F2FC20EEE1ECE5EDE0EE
:101FD40020EDE020EFEEF0F2F32C3130302C3230F3
:101FE400302C3330302C3630302C313230302C32EF
:101FF4003430302C343830302C393630302C3139C0
:102004003230302C33383430302C35373630302CB5
:102014003131353230300A003E532C6B30362C25AA
:1020240062752CCDEEECE5F020F1F2E0EDF6E8E897
:102034000A003E532C6B30372C2562752CC0E4F01B
:10204400E5F120415344550A003C21003C6B3031FA
:102054003D003C6B30323D003C6B30333D003C6B0B
:1020640030343D003C6330313D003C6B30353D0045
:102074003C6B30363D003C6B30373D005265737429
:1020840061727420424C0A0043414E205455204F43
:102094004B0A0043414E205455205265710A0020DA
:1020A40054552054696D654F5554210A00204F4BF7
:1020B4002000204E414B2000205265732043480AE3
:1020C4002000205265732055500A200020444154BA
:1020D40041410A200020545553656C0A20002054C5
:1020E40055455845430A200020444154410A2000E4
:1020F4002053657454696D650A2000204348520AD0
:102104002000205245510A20002054555F4F4B0AAD
:1021140020002054555F4572720A20002054555205
:10212400656164790A2000205455526561647932EE
:102134000A200073656E642074730A0073656E640C
:102144002074734379630A002073656E6420746994
:10215400744379630A20002073656E64207469698E
:102164000A20002073656E642074697453706F7460
:102174000A2000FF1DE4FF1DE9FF1DEEFF1DF2FF15
:0E2184001DF8FF1DFEFF1E02FF1E05FF1E0BB5
:03002300023E1D7D
:0B3E1D00C0E0C083C082C0D075D01888
:103E2800209803023F04C298756801AF99301303C4
:103E3800023F3DD29120113CBFE507D21DD21302AB
:103E48003F04BFA207D216D213023F04BF680DD2A7
:103E580011D218750B00750F00023F04EF64106053
:103E680003023F04D211D219751602750F03750BA0
:103E780000023F3DE50F70078F16050F023F3DE535
:103E88000FB4010FE516B51F05050F023F3DC2111E
:103E9800023F3DE50FB4020AEF646860CEC211022A
:103EA8003F3DE50FB4031E74732510F582E43466B4
:103EB800F583EFF00510250BF50B1516E516707553
:103EC800750F048070E50FB4040DE50BB51F0405EC
:103ED8000F8062C211805EE50F6405701FBF161166
:103EE800D213851016631080531080C211C29180BE
:103EF80044C219C218531080C21180393099363023
:103F0800123190618BE0FFE511C39F4008C212D2C5
:103F18001AC290801ED29074B32511F582E43467DA
:103F2800F583E0F514E50C5214A2D0B3929B8514E6
:053F3800990511C2997A
:093F3D00D0D0D082D083D0E03254
:10416D007BFF7A1E790C1221F4906F58E070147554
:10417D002FFF75301E75317C7BFF7A1E793E122123
:10418D00F48012752FFF75301E75318B7BFF7A1EF3
:10419D00793E1221F47BFF7A1E799A90618CE0F5BD
:1041AD002F1221F47BFF7A1E79C0906101E0F52F6B
:1041BD001221F47BFF7A1E79E7906100E0F52F1252
:1041CD0021F47BFF7A1F790DA210E433F52F122114
:1041DD00F47BFF7A1F79361221F47BFF7A1F796DFC
:1041ED00906410E0F52FA3E0F530906189E0F53192
:1041FD00A3E0F532906187E0F533A3E0F5349066E6
:10420D0024E0F535A3E0F5361221F49068B3E0FE15
:10421D00A3E0FFC3E49FFFE49EFEAB07FA3395E0F6
:10422D00F9F87F007E8C7D0A7C001225ED8F328E91
:10423D00318D308C2F7BFF7A1F79BA1221F47BFFE1
:10424D007A20791C90640FE0F52F1221F47BFF7A10
:0A425D0020793685082F1221F42283
:104267007E207F4D1249DDEF4E70037F0122E490DF
:104277006F58F07E207F501249DDEF4E60151252C5
:10428700EBBF3106906F58740AF0BF3206906F5833
:104297007464F07E207F561249DDEF4E6008124F9E
:1042A7005D90618CEFF07E207F5C1249DDEF4E6000
:1042B70008124F5D906101EFF07E207F621249DDA9
:1042C700EF4E6008124F5D906100EFF07E207F682F
:1042D7001249DDEF4E600D124F5DEC4D4E4F24FF3E
:1042E70092108002C2107E207F6E1249DDEF4E6071
:1042F70023124F5DA804A905AA06AB077F007E8C91
:104307007D0A7C001225ED12267F9068B3EEF0A39C
:10431700EFF0800A9068B374FFF0A374DCF07E209E
:104327007F741249DDEF4E600A124F5D90640FEF04
:10433700F0800690640F7401F07E207F7A1249DDC9
:10434700EF4E6007124F5D8F0880037508017F00ED
:014357002243
:102F9C00E490640FF0906F58F0907080F090708017
:102FAC00E075F003A42477F582E43421F583E493EF
:102FBC00FB740193FA740293F91224EE700302313C
:102FCC0097E4907082F0A3F0907081F0907081E0A3
:102FDC0024E4F582E43469F583E0FF700302318E5A
:102FEC00907080E075F003A42477F582E43421F529
:102FFC0083E493FB740193FA740293F9907082E06A
:10300C00F582758300122507FEEFB5060F907083CD
:10301C007401F0907082E004F0023185907083E0CE
:10302C007003023185EE600302317C907080E0B455
:10303C000700400302318E90304AF8282873023082
:10304C005F0230AC0230E90230EE02305F02311C1C
:10305C0002314C907081E024E4F9E43469FA7B018C
:10306C00C0031B8B2F753000753100E4F532D00393
:10307C001237119070841226BE907084E0F8A3E091
:10308C00F9A3E0FAA3E0FB7F007E8C7D0A7C0012A2
:10309C0025ED12267F9068B3EEF0A3EFF002318E8F
:1030AC00907081E0FD24E4F582E43469F583E0243A
:1030BC00D090618CF074E52DF582E43469F583E0F1
:1030CC0024D0906101F0907081E024E6F582E43424
:1030DC0069F583E024D0906100F002318ED21702A2
:1030EC00318E907081E024E4F9E43469FA7B01C0FC
:1030FC00031B8B2F753000753100E4F532D00312B1
:10310C0037119070841226BE907087E0F50A807299
:10311C00907081E024E4F9E43469FA7B01C0031B6C
:10312C008B2F753000753100E4F532D00312371156
:10313C009070841226BE907087E0906F58F0804299
:10314C00907081E024E4F9E43469FA7B01C0031B3C
:10315C008B2F753000753100E4F532D00312371126
:10316C009070841226BE907087E090640FF08012ED
:10317C00E4907083F0907082F0907081E004F00223
:0B318C002FD8907080E004F0022FA903
:013197002215
:102D8D009069BAE064557004A3E064816064E4F571
:102D9D0011741B2511F582E43466F583E4F0741289
:102DAD002511F582E43466F583E4F074072511F5F9
:102DBD0082E43463F583E4F00511E511B408D2E43F
:102DCD00F51174732511F582E43467F583E4F0058C
:102DDD0011E511B440ECE4F51174BF2511F582E451
:102DED003461F583E4F00511E511B480ECE4F513DD
:102DFD00F512E4907088F0C212C21AC211C213F516
:102E0D001190618BF0F50AF509F510F568C20FC246
:102E1D001CC2179068B374FFF0A374F4F0750CFF27
:102E2D009061007402F0A3F090618CF0906410E456
:102E3D00F0A304F09061897403F0A374E9F090613C
:102E4D0087740BF0A374B9F09066247407F0A37423
:102E5D00D1F0124267EF6003122F9CE4F5179070CA
:102E6D007E7461F0A3748DF090618CE0F517E51719
:102E7D00C394014007E517D394084003E4F517E523
:102E8D0017602890707EE475F00112259B85F08205
:102E9D00F58374C4F0151790707EE475F00112255A
:102EAD009B85F082F583E517F080D4906101E0F504
:102EBD0017E517C394014007E517D394084003E4C1
:102ECD00F517E517602890707EE475F00112259BCB
:102EDD0085F082F58374C8F0151790707EE475F057
:102EED000112259B85F082F583E517F080D4906162
:102EFD0000E0F517E517C394014007E517D39408D3
:102F0D004003E4F517E517602890707EE475F00135
:102F1D0012259B85F082F58374C2F0151790707E93
:102F2D00E475F00112259B85F082F583E517F0809D
:102F3D00D490707EE475F00112259B85F082F583A7
:102F4D00E4F090707E75F00112259B85F082F5837B
:102F5D00E4F0F517C291C290C2ADF5C9D2CDD2CC75
:102F6D00C2C9C2CAF5CDF5CC9068B3E0F5CBA3E0EC
:102F7D00F5CA85CBCD85CACCD29FD29ED29CD2CA62
:0E2F8D00C2ACC298C29975B81075B710D2AC1C
:012F9B002213
:0246CD008F2D2F
:1046CF00E4FF7C617D02FEEEC3952D50120DEDAA25
:1046DF000470010C14F5828A83E02FFF0E80E80D21
:1046EF00EDAA0470010C14F5828A83EFF00DEDAE84
:1046FF000470010C14F5828E837416F0052D052DB0
:10470F007E677FB37C617D02E52DB4040E8F828EB0
:10471F00837410F00FBF00010E80328F828E83746E
:10472F0068F00FBF00010EE52D24FEFB8F828E83F4
:10473F00F00FBF00010E8F828E83EBF00FBF0001D1
:10474F000E8F828E837468F00FBF00010E8C838DE5
:10475F008263A2018E838F8263A201AF2D12363A3C
:0D476F00E52DB4040304FF22E52D2404FF12
:01477C00221A
:1050E6002012351246CD90618BEFF0200A0B7E67B9
:1050F6007FB3E0FDE4FB1245F93017057F0112533B
:1051060056E50A6003F56522E490661AF0F511D2B9
:0951160012C2992099FDD29922E0
:022AD9008F2844
:102ADB0090640FE07003022D8CE54730E712E54A56
:102AEB00B4100D200A077E207F8012443EE4F509C6
:102AFB00E54724BE7003022D5924FA7003022C8182
:102B0B0024046003022D8CE54830E703022BAAE571
:102B1B004A6066E549C394024003022D8CE5497077
:102B2B0007E54A14F5298006E54A241FF529E5290E
:102B3B0075F004A4240FF582746335F0F5837D4C96
:102B4B007F04123628E52975F004A42407F5827456
:102B5B006235F0F5837D507F0412362874FF2549CA
:102B6B00F582E43461F5837481F074BF2529F58215
:102B7B00E43461F5837401F02274122549F582E483
:102B8B003466F583E04480F0E54925E025E02447F1
:102B9B00F582E43466F5837D4C7F0412362822E5FA
:102BAB004B64086003022D8C752801E54A5407FF1E
:102BBB00E528A807088002C333D8FCF5287408253C
:102BCB0013F513B5120674082512F512E54A547F56
:102BDB00FFE549C43354E02FFE74002513F582E45E
:102BEB003460F583EEF0E54AC39480503CEF131349
:102BFB0013541FFFE54925E025E025E025E0244798
:102C0B00F582E43466F583E5822FF582E43583F5AE
:102C1B0083E0FFE528F4FEEF5EF074012513F582E7
:102C2B00E43460F583E4F0803AE54A547FFF1313F4
:102C3B0013541FFFE54925E025E025E025E0244757
:102C4B00F582E43466F583E5822FF582E43583F56E
:102C5B0083E04528F074012513F582E43460F58395
:102C6B007401F074022513F582E43460F5837D4C16
:102C7B007F0612362822E54A54E06440702CE54A60
:102C8B00540F144440FF74072549F582E43463F56F
:102C9B0083EFF0E54925E025E02426F582E4346650
:102CAB00F5837D4C7F041236282274072549F58263
:102CBB00E43463F583E0F55F30E64AE54A131354D9
:102CCB003FFFE55F540FB50714E55F54074480FFE2
:102CDB0074072549F582E43463F583EFF0E54A5434
:102CEB007FFF1313543FFF75F008E549A42FF582BE
:102CFB00E435F0F583E5822473F582E5833467F5DB
:102D0B0083E4F08027E54A547FFF1313543FFF758C
:102D1B00F008E549A42FF582E435F0F583E582242C
:102D2B0073F582E5833467F5837401F075F040E544
:102D3B0049A42412F582E5F03464F583E54A547F07
:102D4B0075F0021226FB7D4CAF4B12362822302732
:102D5B0030E54AB40112200A077E207F8C12443ED4
:102D6B00E54D04907071F022E54AB403149070594C
:102D7B00E0B401037405F0200A077E207F9712440C
:012D8B003E09
:012D8C002224
:1000260030001DC200302718906184E004F0E0D350
:100036009414400C200A077E207FA312443EC22758
:10004600E5157036906646E004F0E05407F0E0FFF0
:100056002407F582E43463F583E0FE30E71C740779
:100066002FF582E43463F583EE547FF074072FF5A1
:1000760082E43463F583E004F515201B2690618540
:10008600E004F0E0543FF0E0FF2473F582E43467C7
:10009600F583E0600ED21B74732FF582E43467F5A6
:1000A60083E4F0201426906623E004F0E0543FF049
:1000B600E0FF24BFF582E43461F583E0600ED214DC
:1000C60074BF2FF582E43461F583E4F020152A909D
:1000D6006186E004F0E05407F0E0FF2412F582E4C4
:1000E6003466F583E0FE30E71074122FF582E434AF
:1000F60066F583EE547FF0D215201303020A1DE540
:100106001654802473F582E43466AF82F5298F2A6B
:10011600301D0CC21D200A077E207FB112443E30DE
:10012600160CC216200A077E207FB612443E2018FF
:1001360006201903020A1B852A82852983A3E0FF6C
:1001460090640FE0FEEF6E6003020A17E52A2407AB
:10015600F582E43529F583E0FEE52A2406F582E4F6
:100166003529F583E07C002400F52CEC3EF52B8543
:100176002A82852983E0544F24BF603E24FE6054C2
:100186001470030202B924FB7003020416147003F0
:10019600020436147003020436240B6003020A17A5
:1001A600200A077E207FBC12443EE50C54E5F52864
:1001B600A2D0929B7599E5020A17200A077E207F36
:1001C600C612443EE50C54E5F528A2D0929B7599DB
:1001D600E5020A17200A077E207FD012443EE50C6E
:1001E60054E5F528A2D0929B7599E5852A82852942
:1001F60083A3A3E0642D6003020A17852983852A59
:100206008263A20190666763A2017F0A12363AE50D
:100216002A2404F582E43529F583E0543F64066018
:10022600030202B4E52A2408F582E43529F583E0C1
:1002360030E75A200A077E207FD912443E30270332
:10024600020A17D227E4907059F0906184F0906604
:1002560024E0FEA3E0FFC3E52C9FFDE52B9EC4F83A
:1002660054F0C868EDC4540F4890705AF0ED540F1E
:1002760025E0FFE433E52A2408F582E43529F583F1
:10028600E0640154012F90705FF0020A17200A07FC
:100296007E207FE212443E202703020A17907059FF
:1002A600E064066003020A177402F0020A17C22706
:1002B600020A17200A077E207FEC12443E852A8216
:1002C600852983A3A3E06467600302036F200A07FE
:1002D6007E207FF412443E75090AE52A2408F58239
:1002E600E43529F583E0750D00F50EE52A2409F5B8
:1002F60082E43529F583E0FEE4EE420DE52A240A80
:10030600F582E43529F583E0F55FE52A240BF582CD
:10031600E43529F583E0F55EE52A240CF582E4351B
:1003260029F583E0F55DE52A240DF582E43529F506
:1003360083E0F560E52A240EF582E43529F583E0AD
:10034600F55BAE0DAF0E7C037DE81225468F5C1281
:100356003F4690705BE564F0A3E563F0A3E562F0C9
:10036600A3E561F0D229020A17852A82852983A38B
:10037600A3E0642D6003020A17852983852A826318
:10038600A20190666763A2017F0A12363AE52A2423
:1003960004F582E43529F583E0543F6406706CE584
:1003A6002A2408F582E43529F583E0FD30E7453057
:1003B6002703020A17D227E4907059F0907071F063
:1003C600906624E0FEA3E0FFC3E52C9FFBE52B9E91
:1003D600C4F854F0C868EBC4540F4890705AF0EB58
:1003E600540F25E0FFE433ED640154012F90705F54
:1003F600F0020A17202703020A17907059E06406D4
:100406006003020A177402F0020A17C227020A17CB
:10041600200A077E207FFF12443E906102740BF093
:1004260090640FE0906103F07F021250E6020A1713
:10043600200A077E217F0612443EE509C394055033
:10044600050509020A17202703020539907071E095
:10045600FF60686401702E200A077E217F0D12441A
:100466003E90666763A20190610263A2017F091252
:10047600363A9061027408F0906106740AF07F09BA
:100486001250E6802C200A077E217F1612443E90E9
:10049600666763A20190610263A2017F0912363A80
:1004A6009061027408F09061067447F07F0912505B
:1004B600E6E4907071F0C227020A17907059E06462
:1004C600057034200A077E217F2012443E9066671D
:1004D60063A20190610263A2017F0912363A90611C
:1004E600027408F090610614F07F091250E69070CD
:1004F600597406F0020A17907059E06403703420AC
:100506000A077E217F2B12443E90666763A2019004
:10051600610263A2017F0912363A9061027408F003
:1005260090610614F07F091250E69070597407F036
:10053600020A17E51365127003020627E51224085E
:10054600F52874082512F512D21C9061027408F081
:1005560090640FE0906103F0A3741EF0A37401F0A1
:10056600A37403F0A3E508F0906411E0FF7400257E
:1005760028F582E43460F583E0FE2F906108F0EE02
:10058600FF906411E02F906410E03400FF3395E093
:10059600906109EFF074012528F582E43460F58353
:1005A600E090610AF074022528F582E43460F58350
:1005B600E0F56474032528F582E43460F583E0F5FC
:1005C6006374042528F582E43460F583E0F56274EB
:1005D600052528F582E43460F583E0F561123CE8F0
:1005E600AF5C7E007C037DE81225348E0D8F0EEF06
:1005F60090610BF0E50DA3F0A3E55FF0A3E55EF0D7
:10060600A3E55DF0A3E560F0A3E55BF07F10125073
:10061600E6300A03020A177E217F3712443E020A99
:10062600172015030206E3C2159061027408F090C4
:10063600640FE0906103F0A37407F0A37401F0A3C4
:10064600F0A3E508F0906411E0FF906186E0FEC437
:100656003354E02F906108F0EE75F020A4FF90640B
:1006660011E02F906410E035F0FF3395E0906109BA
:10067600EFF0906186E0FF25E025E02447F582E46F
:100686003466F583E090610AF0EF25E025E0244822
:10069600F582E43466F583E090610BF0906186E0C4
:1006A60025E025E02449F582E43466F583E090618F
:1006B6000CF0EF25E025E0244AF582E43466F58364
:1006C600E090610DF0E4A3F07F0D1250E6300A03CE
:1006D600020A177E217F4012443E020A17E5157072
:1006E60003020855200A077E217F4C12443EE51579
:1006F60025E025E0F55FE4F5159061027408F090B9
:10070600640FE0906103F0A37422F0E55F2480A3F8
:10071600F0A37401F0A3E508F090618AE0FF90660B
:1007260046E0FEC43354E02F906108F0EE75F020E9
:10073600A4FF90618AE02F906189E035F0FF339540
:10074600E0906109EFF0906646E075F040A424124F
:10075600F582E5F03464F58363A20190610A63A231
:1007660001AF5F12364AE55F75F003A42408F52849
:10077600906646E0FF25E025E02426F582E434660F
:10078600F583E0F564EF25E025E02427F582E434DF
:1007960066F583E0F563906646E0FF25E025E024F4
:1007A60028F582E43466F583E0F562EF25E025E07E
:1007B6002429F582E43466F583E0F561123CE8AF5E
:1007C6005C7E007C037DE81225348E0D8F0EEFAE25
:1007D60028052874022EF582E43461F583EFF0E5EE
:1007E6000DFFAE28052874022EF582E43461F583E8
:1007F600EFF0AF28052874022FF582E43461F58303
:10080600E55FF0AF28052874022FF582E43461F520
:1008160083E55EF0AF28052874022FF582E4346183
:10082600F583E55DF0AF28052874022FF582E434E0
:1008360061F583E560F0AF28052874022FF582E4A0
:100846003461F583E55BF0AF281250E6020A172003
:100856001403020980200A077E217F5B12443EC2F0
:10086600149061027408F090640FE0906103F0A3A5
:100876007425F0A37401F0A3F0A3E508F090618855
:10088600E0FF906623E0FE2F906108F0EEFF906196
:1008960088E02F906187E03400FF3395E09061098E
:1008A600EFF0906623E025E025E0F528FF052874A3
:1008B6000F2FF582E43463F583E090610AF0AF28E8
:1008C6000528740F2FF582E43463F583E090610BFD
:1008D600F0AF280528740F2FF582E43463F583E022
:1008E60090610CF0AF280528740F2FF582E434636D
:1008F600F583E090610DF0E4A3F074FC2528F5285B
:10090600FF052874072FF582E43462F583E0F56469
:10091600AF28052874072FF582E43462F583E0F5E5
:1009260063AF28052874072FF582E43462F583E067
:10093600F562AF28052874072FF582E43462F58343
:10094600E0F561123CE8AF5C7E007C037DE8122591
:10095600348E0D8F0EEF90610FF0E50DA3F0A3E539
:100966005FF0A3E55EF0A3E55DF0A3E560F0A3E527
:100976005BF07F141250E6020A17201B03020A04DA
:10098600200A077E217F6712443EC21B90610274D3
:1009960008F090640FE0906103F0A37409F0A3746B
:1009A60084F0A37403F0A3E508F090618AE0FF9059
:1009B6006185E0FE25E025E02F906108F0EE75F0F8
:1009C60004A4FF90618AE02F906189E035F0FF333F
:1009D60095E0906109EFF0906185E075F008A42438
:1009E60012F582E5F03464F58363A20190610A632F
:1009F600A2017F0412364A7F141250E680139061DA
:100A0600027409F090640FE0906103F07F021250C7
:070A1600E6C219C218C21369
:010A1D0022B6
:0100220022BB
:10495D00021279E493A3F8E493A34003F68001F2E5
:10496D0008DFF48029E493A3F85407240CC8C3335B
:10497D00C4540F4420C8834004F456800146F6DF2A
:10498D00E4800B010204081020408090535FE47E08
:10499D00019360BCA3FF543F30E509541FFEE4931F
:1049AD00A360010ECF54C025E060A840B8E493A3E6
:1049BD00FAE493A3F8E493A3C8C582C8CAC583CA11
:1049CD00F0A3C8C582C8CAC583CADFE9DEE780BEC9
:015365000047
:1024EE00BB010689828A83E0225002E722BBFE02EC
:0924FE00E32289828A83E493221F
:10250700BB010CE58229F582E5833AF583E0225089
:1025170006E92582F8E622BBFE06E92582F8E222D3
:0D252700E58229F582E5833AF583E49322ED
:10253400EF8DF0A4A8F0CF8CF0A428CE8DF0A42EBB
:02254400FE2275
:10254600BC000BBE0029EF8DF084FFADF022E4CC79
:10255600F875F008EF2FFFEE33FEEC33FCEE9DEC42
:10256600984005FCEE9DFE0FD5F0E9E4CEFD22ED88
:10257600F8F5F0EE8420D21CFEADF075F008EF2FD2
:10258600FFED33FD4007985006D5F0F222C398FDC3
:052596000FD5F0EA2260
:10259B00A3F8E0C5F025F0F0E582158270021583F3
:0625AB00E0C838F0E82250
:1025B10075F008758200EF2FFFEE33FECD33CDCCE1
:1025C10033CCC58233C5829BED9AEC99E582984064
:1025D1000CF582EE9BFEED9AFDEC99FC0FD5F0D641
:1025E100E4CEFBE4CDFAE4CCF9A88222B800C1B96B
:1025F1000059BA002DEC8BF084CFCECDFCE5F0CBA9
:10260100F97818EF2FFFEE33FEED33FDEC33FCEBE1
:1026110033FB10D703994004EB99FB0FD8E5E4F99C
:10262100FA227818EF2FFFEE33FEED33FDEC33FC89
:10263100C933C910D7059BE99A4007EC9BFCE99A7D
:10264100F90FD8E0E4C9FAE4CCFB2275F010EF2FC2
:10265100FFEE33FEED33FDCC33CCC833C810D707C2
:102661009BEC9AE899400AED9BFDEC9AFCE899F8FD
:0E2671000FD5F0DAE4CDFBE4CCFAE4C8F92290
:0E267F00C3E49FFFE49EFEE49DFDE49CFC226C
:10268D00EB9FF5F0EA9E42F0E99D42F0E89C45F0A3
:01269D00221A
:10269E00E493FC740193FD740293FE740393FF2282
:1026AE00E493F8740193F9740293FA740393FB2282
:0C26BE00ECF0A3EDF0A3EEF0A3EFF0228F
:1026CA00A8828583F0D083D0821226E11226E112F5
:1026DA0026E11226E1E473E493A3C583C5F0C5831A
:1026EA00C8C582C8F0A3C583C5F0C583C8C582C85A
:0126FA0022BD
:0C26FB00A42582F582E5F03583F58322EA
:10219200E53B242FF8E6053B22782C302502782FE8
:1021A200E475F0011227680224EE201EEB7F2ED286
:1021B2001E8018EF540F2490D43440D4FF30220BE9
:1021C200EF24BFB41A0050032461FFE53C600215FE
:1021D2003C053FE53F7002053E30250D782CE47545
:1021E200F001122768EF0227070250137403D22569
:1021F2008003E4C225F53B8B2C8A2D892EE4F53C25
:10220200F53EF53FE53C60077F201221CD80F57554
:102212003DFFC21FC21EC220C221C223C224C22647
:1022220012219BFF700D3025057F001221DEAF3F8A
:10223200AE3E22B4255FC2D5C22212219BFF24D01A
:10224200B40A00501A75F00A783C30D50508B6FF7A
:102252000106C6A426F620D5047002D22180D92414
:10226200CFB41A00EF5004C2E5D2220223DED21FFD
:1022720080C6D21E80C0D22080BCD2D580BAD223E2
:1022820080B47F201221CD2020077401B53C00408C
:10229200F1122192FF1221CD022206D226D22480EF
:1022A20095122192FB122192FA122192F94A4B7055
:1022B2000679AF7A247BFF20202EE53C602A7E003F
:1022C2008E8275830012250760060EEE653D70F062
:1022D200C2D5EBC0E0EAC0E0E9C0E0EE122425D0AE
:1022E200E0F9D0E0FAD0E0FB1224EEFF60AAEBC0E6
:1022F200E0EAC0E0E9C0E01221CDD0E02401F9D04B
:10230200E03400FAD0E0FBE53D0460DCD53DD98045
:10231200877BFF7A247921D220809C7910800279F0
:1023220008C224C2268008D2D5790A8004790AC25A
:10233200D5E53D047002F53DE4FAFDFEFF1221925F
:10234200FC7B08201F13122192FD7B10301E0A1203
:102352002192FE122192FF7B20EC3382D592D5503E
:1023620013C3E4301E069FFFE49EFEE4201F039D7C
:10237200FDE49CFCE4CBF8C21FEC700CCFCECDCCBC
:10238200E824F8F870F38017C3EF33FFEE33FEED65
:1023920033FDEC33FCEB33FB994002FB0FD8E9EB46
:1023A200301F05F8D0E0C448B21FC0E00AEC4D4E21
:1023B2004F78207B0070C2EAB53D0040BCC0E012FD
:1023C2002427D0F0D0E0201F04C4C0E0C4B21FC054
:1023D200F01221B6D0F0D5F0EB0222061227C72266
:1023E200A353231D5822744C22704223214F2329C8
:0F23F20044232949228943232F552313462313BC
:102401004523134724CF5022782D227C2E229F2B47
:10241100228023229D2024B82A22384800002297B6
:102421003F3F3F00790AA2D5202114302309B9107A
:10243100020404B9080104A2D52024025001042099
:1024410020689220B53C005034C0E07F2030211933
:102451007F30A22072247223500F12247EC220C228
:1024610024C223C2267F30800F302303E9C0E0124B
:1024710021CD302303D0E0F9D0E0B53CCC30231797
:102481007F30B9100C1221CD7F583022077F788020
:1024910003B908031221CD3020057F2D0221CD7F04
:1024A100202026F87F2B2024F322922080CF286E33
:1024B100756C6C2900D21F122192301FF8C21F784F
:1024C1003C30D50108F60222382D504349581221DB
:1024D100922403B405004001E49024CA931221BE62
:0D24E100743A1221BED221753C0402231D65
:103711008B2C8A2D892EE4F538F537F536F535F5FC
:1037210033F534E5304531452F6012EBC0E0EAC096
:10373100E0E9C0E0AB2FAA30A931122778AB2C0504
:103741002EE52EAA2D7002052D14F91224EEF5395D
:10375100C394094007E539D3940D40E1E53964206C
:1037610060DBE539B42D054334038016E539B42B0C
:1037710005433401800C74FF252EF52E74FF352D81
:10378100F52DE53260046410703FAB2CAA2DA92EF3
:103791001224EE64306009E532702E75320A8029F8
:1037A100900001122507FF64786004EFB4581343B9
:1037B10034017532107402252EF52EE4352DF52DC8
:1037C1008007E5327003753208AB2C052EE52EAA71
:1037D1002D7002052D14F91224EEF539C3946140C0
:1037E1000AE539D3947A50035339DF74D02539F57A
:1037F10039C3940A400CE5399411406D74F92539A7
:10380100F539E539D39532506043340185383D852A
:10381100373C85363B85353AAF327E00E4FCFDAB63
:1038210038AA37A936A835122719C8ECC8C9EDC975
:10383100CAEECACBEFCBE4FCFDFEEB2539F538EE41
:103841003AF537ED39F536EC38F535AF38AE37ADF9
:1038510036FCAB3DAA3CA93BA83AD312268D5003B6
:103861000237CA4334040237CAE53420E003E48056
:103871002DE5304531452F601EAB2CE52E24FFF997
:10388100E52D34FFFAEBC0E0EAC0E0E9C0E0AB2F80
:10389100AA30A931122778E53430E20774FFFFFE20
:1038A100FDFC22E534AF38AE37AD36AC3530E1033F
:0438B10002267F224A
:10270700BB010689828A83F0225002F722BBFE01B1
:02271700F322AB
:10271900E88FF0A4CC8BF0A42CFCE98EF0A42CFC5F
:102729008AF0EDA42CFCEA8EF0A4CDA8F08BF0A4DD
:102739002DCC3825F0FDE98FF0A42CCD35F0FCEB3C
:102749008EF0A4FEA9F0EB8FF0A4CFC5F02ECD3901
:0F275900FEE43CFCEAA42DCE35F0FDE43CFC226E
:10276800FAE6FB0808E6F925F0F618E6CA3AF62272
:10277800BB011A89828A83D0F0D0E0F8D0E0F9D082
:10278800E0FAD0E0FBE8C0E0C0F00227F65016E916
:10279800F8D083D082D0E0F9D0E0FAD0E0FBC08254
:1027A800C0830227EDBBFE16E9F8D083D082D0E0C3
:0F27B800F9D0E0FAD0E0FBC082C0830227FF22F5
:1027C700D083D082F8E4937012740193700DA3A3A1
:1027D70093F8740193F5828883E4737402936860B5
:0627E700EFA3A3A380DFB5
:0927ED00EBF608EAF608E9F62211
:0927F600EBF0A3EAF0A3E9F022E4
:0927FF00EBF208EAF208E9F2220B
:00000001FF
